:100000003EC1000058C1000056C1000054C10000AC
:1000100052C1000050C100004EC100004CC10000A0
:100020004AC1000048C1000046C100000C94680BA2
:1000300042C1000040C100003EC100003CC10000C0
:100040003AC1000038C1000036C1000034C10000D0
:1000500032C1000030C100002EC100002CC10000E0
:100060002AC1000028C1000026C1000024C10000F0
:1000700022C10000DE02E302EE02F802FE020403E7
:1000800030033C034103460355035A0365038403CD
:1000900098039E03A603AC03B203BA030B04270420
:1000A00038044304480544054C0550054A054605F7
:1000B0004E055205330C530C390D530C390D950C6C
:1000C000B70C390D0A0D1C0D2203690062006D008A
:1000D0002D00630061007000730065006E00730006
:1000E00065002D00750073006200000022035400BB
:1000F0006F006D00200057006F006E0067002D003C
:1001000043006F0072006E0061006C006C00000024
:10011000040309040902540003010080FA090400E1
:10012000000103010100092111010001222500073E
:1001300005810308000A0904010001030000000909
:1001400021110100012220000705830308000A098C
:10015000040200010300000009211101000122BE78
:10016000000705820319000A120110010000002097
:10017000810402000100010200010600FF0901A143
:10018000010902150025FF7508950881020903156C
:100190000025FF750895089102C005010906A10117
:1001A0000508190129031500250195037501910220
:1001B000950175059101050719E029E7150025014D
:1001C00095087501810205071900293115002501DF
:1001D0009532750181029501750181010507193379
:1001E000299B15002501956975018102950175010D
:1001F00081010507199D29A41500250195087501A0
:1002000081020501198129831500250195037501D6
:100210008102050C19B029B8150025019509750151
:100220008102050C09CD09E209E909EA0A8A010AF5
:1002300092010A94010A21020A23020A24020A25D1
:10024000020A27020A2A0215002501950D7501816F
:1002500002950175028101C005010906A101750120
:100260009508810195017508810195057501910138
:10027000950175039101950675088101C00011244F
:100280001FBECFEFD4E0DEBFCDBF11E0A0E0B1E0F4
:10029000ECEBFFE102C005900D92A635B107D9F74E
:1002A00013E0A6E5B1E001C01D92A837B107E1F760
:1002B0008DD00C94DC0FA4CE80E291E00E949E0EC3
:1002C00080E191E00E949E0E80E091E00E949E0EEF
:1002D000E2EEF0E0808184608083EAC280E291E017
:1002E0000E946E0D80E191E00E946E0D80E091E031
:1002F0000C946E0D80912E0190912F01009729F0A2
:10030000019790932F0180932E0180911E0190916F
:100310001F01009729F0019790931F0180931E0100
:1003200080910E0190910F01009729F00197909311
:100330000F0180930E01CAC20F931F93CF93DF93D7
:10034000FC01C901E80121E0E032F20711F433D3E6
:1003500005C021E0E031F20721F4BCD188E090E053
:1003600005C066817781B9D389E190E0998388835C
:1003700080E0DF91CF911F910F910895AC01C901E9
:1003800021E04032520709F482C44051514009F43F
:1003900009C180C484B7877F84BF88E10FB6F89411
:1003A00080936000109260000FBE90E080E80FB66E
:1003B000F89480936100909361000FBE2BD022D7F8
:1003C00072D225D7479A47980C94590BE3DF78945B
:1003D000E3D2EFD575D6C8D28FE19EE40197F1F74D
:1003E00000C000003AD0809184019091850101966F
:1003F00009F411D552D480E291E00E94B10E80E15F
:1004000091E00E94B10E80E091E00E94B10E0E9446
:10041000520DF0CFE8D6289A0895CF93DF939093AA
:100420008501809384012898EC01CC0FDD1FCC0F4F
:10043000DD1F8D2FE1D68C2FDFD6289ADF91CF914B
:1004400008956091840180E090E00E94CA0F60915D
:10045000850181E090E00C94CA0FCF93DF9381E097
:1004600090E00E94B30FC82FD0E0DC2FCC2780E0B3
:1004700090E00E94B30F9E01282BC901DF91CF911C
:10048000CCCF292F332723303105A9F06CF421304C
:10049000310509F442C02230310509F043C084E53A
:1004A00090E024E131E042C021323105C9F022322E
:1004B000310519F137C099278130910541F082301B
:1004C000910541F0892B71F5E0E1F1E005C0ECEE1A
:1004D000F0E002C0E8ECF0E0849190E09F0126C0DB
:1004E000633000F5E62FF0E0EE0FFF1FE25CFE4FF9
:1004F0002081318189E090E019C0633098F4E62FC3
:10050000F0E0DF01AA0FBB1FA85CBE4F2D913C910C
:10051000EB5CFE4F808190E009C082E190E028E62C
:1005200031E004C080E090E020E030E0FA01318367
:1005300020830895EF92FF920F931F93CF93DF9341
:1005400051E0EE24E394F12C461728F1E62FF0E079
:10055000EE0FFF1FEE0FFF1FE757FE4F20E030E0CA
:10056000DC01A50FB11D8F01020F131FE801788177
:1005700073304CF07C918701022E01C0000F0A9469
:10058000EAF7702B7C932F5F3F4F2430310559F7EA
:100590006F5F5F5FD9CFDF91CF911F910F91FF9078
:1005A000EF900895DC014C9150E04D30510508F07A
:1005B00090C0465C5F4FFA010C94800F11968C91AD
:1005C00080933201089511962C91119712968C9177
:1005D00090E0982F8827820F911D1FCF11968C9144
:1005E000882309F476C0E0913301F0913401099435
:1005F00011968C91882309F46CC023CF11968C91AD
:10060000882309F466C007C413963C911397129689
:100610002C9112971196AC91EA2FEF73E73108F005
:1006200058C0243008F055C0A295A695A695A37091
:10063000A150A33040F4B0E0AA0FBB1FAC5BBE4F8B
:100640008D919C9102C080E592E0F0E0EE0FFF1FDB
:10065000EE0FFF1FE20FF11DE80FF91F3083089521
:1006600012968C9112971196EC91E83090F5F0E08B
:10067000E85FFC4F8083089511968C91882349F19F
:100680001FC511968C91882321F135C513968C9145
:10069000139712969C91129711962C912093870193
:1006A000909386018093880103C111968C918823D1
:1006B00081F048C111968D919D91AC918093E50197
:1006C0009093E601A093E701089511968C91811112
:1006D00069C408950F931F93CF93DF938C0188E033
:1006E000D8011D928A95E9F740913201F8014083C3
:1006F00050E0415051094B30510508F0CFC0495BE3
:100700005F4FFA010C94800F84E0D80111968C930E
:10071000119798E012969C93129797E113969C93E9
:10072000139714968C93149781E015968C93B6C00A
:1007300046E060E0C801FEDE83E005C04DE067E012
:10074000C801F8DE84E080933201A8C044E16EE085
:10075000C801F0DE85E0F7CF47E165E1C801EADED8
:1007600082E0F1CF9091840180918501F80191831D
:10077000828394C05091810140918001852F8295A0
:10078000880F880F807C842BD80111968C93F801F8
:100790003296842F90E0880F991F880F991F20911F
:1007A000300130913101280F391F80E090E0D901EC
:1007B000A80FB91F6C916193019684309105B9F728
:1007C0004F5F40938001473109F068C0109280016B
:1007D00081E0850F843019F08093810102C010926E
:1007E000810180918101813061F040F0823061F0BF
:1007F000833009F053C08CEA92E008C080E592E0B3
:1008000005C080E193E002C084EF91E09093310154
:100810008093300143C080917F01F8018183A82F2C
:10082000B0E0AA0FBB1FAA0FBB1FA85FBC4F4D9122
:100830005D916D917C9142835383648375838F5F57
:1008400080937F01823051F510927F0127C0A0E58F
:10085000B1E0E801219681E08F5F9D919993992302
:1008600011F08730C9F7F801E80FF11D108216C0AA
:1008700080918701F8018183809186018283809134
:10088000880183830BC02091E5013091E6014091FE
:10089000E701D80111962D933D934C93DF91CF91B1
:1008A0001F910F910895249A259A269A279A0895C0
:1008B000109283012C982D982E982F988091870163
:1008C000813019F42F9A109282010895809183014A
:1008D0008F3F19F08F5F8093830180918701813072
:1008E000B1F49091830180918601981302C02E98F3
:1008F000089580918201882351F0209188019217F8
:1009000030F0109283018150809382012E9A0895D5
:10091000809182018F5F8093820108959091870179
:10092000923079F480FF02C02D9A01C02D9881FF8A
:1009300002C02E9A01C02E9882FF02C02C9A089500
:100940002C980895609187018AE791E00E94CA0F70
:10095000609186018BE791E00E94CA0F6091880147
:100960008CE791E00C94CA0F8AE791E00E94B30FE4
:10097000833018F48093870102C0109287018BE7BF
:1009800091E00E94B30F809386018CE791E00E9472
:10099000B30F8093880108958CE5E9E8F1E0DF0169
:1009A0001D928A95E9F78CE0E8EEF1E0DF011D92F7
:1009B0008A95E9F708958F929F92AF92BF92DF9246
:1009C000EF92FF920F931F93CF93DF93EC01AED37F
:1009D0008150833048F4E82FF0E0EE0FFF1FE65B14
:1009E000FE4FA081B18102C0A0E5B2E020E030E07E
:1009F000F12C01E010E0490195948794DF2C80E010
:100A000090E0A40148515E4F4A01522F5170E52EEB
:100A1000F5E0FF1508F44EC0F401608170E0EE20AF
:100A200059F0AC014C5F5F4F580102C0AA0CBB1CCF
:100A30004A95E2F7A50107C0A801082E02C0440F9D
:100A4000551F0A94E2F746235723452B69F1AD0160
:100A5000480F591FFA014081443030F150E3540FE0
:100A6000533010F1F394BE016D0D711DFB014283F3
:100A700050E0405E510948305105B0F44E5A5F4F86
:100A80006881FA010C94800F6E5F0DC0605E0BC030
:100A90006F5F09C0605F07C06C5F05C0605C03C02A
:100AA000685F01C06058688301968430910511F039
:100AB000DF2CAECF2F5F3F4F14962731310509F061
:100AC0009ACFDF91CF911F910F91FF90EF90DF9020
:100AD000BF90AF909F908F9008952F923F924F922A
:100AE0005F926F927F928F929F92AF92BF92CF92BE
:100AF000DF92EF92FF920F931F93CF93DF9300D07B
:100B00001F92CDB7DEB79B838A835B010FD38150E1
:100B1000833048F4E82FF0E0EE0FFF1FE65BFE4F56
:100B20008081918102C080E592E03C01E12CF12CB2
:100B300088248394912C6701D594C79400E010E039
:100B4000C60188519E4F6C019E2D9170392EF60181
:100B5000208130E0332051F0C8010496A40102C086
:100B6000440F551F8A95E2F7CA0107C0C401002E41
:100B700002C0880F991F0A94E2F782239323892BDE
:100B800009F456C0F301E00FF11F2081213E99F0D6
:100B900060F4233D38F4203D08F04AC0233008F4C7
:100BA00047C025C0203EB1F022C0253E21F090F084
:100BB000283EE8F40FC0F501808190E030E2320F6A
:100BC00002C0959587953A95E2F780FD03C0298389
:100BD0009FDE2981205EC401022E01C0880F0A9485
:100BE000EAF7EA81FB819081982B908321C0422E05
:100BF000469446944694512C2770222EF501E40D1C
:100C0000F51D818190E0022E02C0959587950A948A
:100C1000E2F780FF7DDEEA81FB81E40DF51DC40172
:100C2000022C01C0880F0A94EAF79181982B9183D6
:100C30000F5F1F4F0430110509F089CFFFEFEF1A46
:100C4000FF0A44E0640E711C57E1E516F10409F057
:100C500072CFEA81FB818181887F8183838D887F48
:100C6000838F0F900F900F90DF91CF911F910F9175
:100C7000FF90EF90DF90CF90BF90AF909F908F90BC
:100C80007F906F905F904F903F902F900895FC0160
:100C9000808144CEFC01808141CE4F925F926F9261
:100CA0007F928F929F92AF92BF92CF92DF92EF92FC
:100CB000FF920F931F93CF93DF9300D000D0CDB757
:100CC000DEB78CE0E8EEF1E0DF011D928A95E9F7EE
:100CD00069E8E62E61E0F62E00E010E09924939496
:100CE00075E0A72EDD24D394E8ECBE2EC02EE02FB5
:100CF000E695E695E695F0E0EB51FE4F808190E0B9
:100D0000202F277002C0959587952A95E2F780FDE0
:100D100064C0802F84D2479A479819821A821B8216
:100D20001C82892D8A95F1F74899998249999A826E
:100D30004A999B824B999C82980135952795AE01E3
:100D40004F5F5F4F2701D70180E090E028513E4F71
:100D5000EC2DE1707E2E682EFA016191AF01F20157
:100D6000662319F06081615002C060816F5F60830B
:100D7000BD018C9087FE02C01C9204C0F5E0F815FE
:100D80000CF4AC921196FB0160816330B4F0F90170
:100D90008080772051F0BC016C5F7F4FFD2D01C03A
:100DA000FF0F6A95EAF76F2F05C06D2D01C0660F22
:100DB0006A94EAF76829F90160830196FFEF4F1AF8
:100DC0005F0A8430910539F622D2479A479866E146
:100DD000C61619F08B2D8A95F1F70F5F1F4F84E02F
:100DE000E80EF11C0731110509F080CF0F900F902C
:100DF0000F900F90DF91CF911F910F91FF90EF9087
:100E0000DF90CF90BF90AF909F908F907F906F902A
:100E10005F904F900895AF92BF92CF92DF92EF9282
:100E2000FF920F931F93CF93DF9320E532E0F12CD5
:100E3000B12C80E090E0F901E80FF91F40814130CA
:100E400021F0423019F4B39401C0F3940196843038
:100E5000910589F72C5F3F4F82E02C3A380749F71C
:100E6000C0E0D0E0CC24CA9423E0D22E00E010E011
:100E7000C601801B910B82309105C0F1EC01D69523
:100E8000C795C00FD11FCE01C8DA8FE891E0019756
:100E9000F1F700C0000090E2E92EFFDEEA94E9F7E6
:100EA00029E831E040E552E060E080E090E0F901BF
:100EB000E80FF91F708173303CF0FA01E80FF91F59
:100EC0007081743008F06F5F01968430910579F776
:100ED0002C5F3F4F4C5F5F4F91E0253E390729F76C
:100EE0006B1510F48E01C4CF6E01C2CF6E010FEFEF
:100EF00013E0A12CB12CC8018A199B0982309105FD
:100F0000C0F1EC01D695C795CA0DDB1DCE0185DA7F
:100F10008FE891E00197F1F700C00000B0E2EB2EFE
:100F2000BCDEEA94E9F749E851E080E592E060E050
:100F300020E030E0FA01E20FF31F708173303CF0E3
:100F4000FC01E20FF31F7081713009F46F5F2F5FB6
:100F50003F4F2430310571F74C5F5F4F049621E01D
:100F6000453E520729F76F1510F45E01C4CF8E017C
:100F7000C2CFC6018C1B9D0BF4E096958795FA9520
:100F8000E1F76FE070E0ABD78C0F9D1F46DADF9181
:100F9000CF911F910F91FF90EF90DF90CF90BF9076
:100FA000AF9086CC43E050E06DE771E085EE91E0D4
:100FB000E2C743E050E06DE771E085EE91E0C3D712
:100FC0008091E5018F3F71F48091E6018F3F51F4EC
:100FD0008091E7018F3F31F41092E5011092E60114
:100FE0001092E70108958F929F92AF92BF92CF9295
:100FF000DF92EF92FF920F931F93CF93DF936C01D9
:101000004B01C0E0D0E07401EC0EFD1E00E010E0EA
:101010005601AC0EBD1EC8018A0D9B1DA4D78F3F83
:1010200009F480E0F70181937F010F5F1F4F0430C7
:10103000110589F72496CC35D10529F7DF91CF9199
:101040001F910F91FF90EF90DF90CF90BF90AF90E6
:101050009F908F9008958F929F92AF92BF92CF9260
:10106000DF92EF92FF920F931F93CF93DF936C0168
:101070004B01C0E0D0E07401EC0EFD1E00E010E07A
:101080005601AC0EBD1EF70161917F01C8018A0DAA
:101090009B1D80D70F5F1F4F04301105A1F72496C9
:1010A000CC35D10541F7DF91CF911F910F91FF9082
:1010B000EF90DF90CF90BF90AF909F908F9008956A
:1010C00048E050E062E771E088E093E03CD760E5FB
:1010D00072E082E090E087DF60E173E08EE590E00F
:1010E00082DF64EF71E08AEB90E07DDF6CEA72E012
:1010F00086E191E078CF48E050E062E771E088E077
:1011000093E039D760E572E082E090E0A4DF60E12F
:1011100073E08EE590E09FDF64EF71E08AEB90E092
:101120009ADF6CEA72E086E191E095CF0F931F930E
:10113000CF93DF9340E552E020E030E0C0E061E093
:1011400070E0F901F595E795E851FE4FA081B0E018
:1011500080E090E0D22FD170DD2351F0FC01349675
:101160008B0102C0000F111FEA95E2F7F80107C0DA
:10117000FB01082E02C0EE0FFF1F0A94E2F7EA23DC
:10118000FB23EF2B79F0FA01E80FF91FE081E13D35
:1011900031F0E23D31F0E03D29F4C16003C0C260AE
:1011A00001C0C460019684309105B1F62F5F3F4FB6
:1011B0004C5F5F4F2731310521F6CC2371F0E8E019
:1011C000F3E08191982F92959F709C1302C08F70CD
:1011D00005C013E0E031F107A1F780E0DF91CF9186
:1011E0001F910F910895219A209A229A84E58CBD2F
:1011F0008DB581608DBD08958EBD0DB407FEFDCF08
:101200008EB508953C9A3D9A3E9A3F9A0895459826
:10121000449888E1459A45988150E1F708954598AA
:101220004498449A459A4598449890E0981721F03C
:10123000459A45989F5FFACF0895CF92DF92EF923B
:10124000FF920F931F93CF93DF937C018B01EA01F1
:10125000C9D1811131C0209731F088819981081B53
:10126000190BE80EF91EC12CD12C0115110519F12D
:101270008091E80085FD14C08091E8008E7780930E
:10128000E80010D4209741F0888199818C0D9D1D34
:101290009983888385E010C0A5D1882331F30CC0E1
:1012A000F70181917F018093F10001501109FFEF57
:1012B000CF1ADF0ADACF80E0DF91CF911F910F9133
:1012C000FF90EF90DF90CF900895209176033091BA
:1012D00077032617370748F06115710539F4209117
:1012E000E8002E772093E80001C0B90120E06115E5
:1012F0007105D1F130916F03332309F441C03530CA
:1013000009F440C03091E80033FD38C03091E80066
:1013100032FF06C08091E80082FF29C080E0089576
:101320003091E80030FFE3CF2091F20030E0FC0183
:10133000281B390BCF01820F931F6115710549F0EE
:101340008032910530F481918093F10061507109F0
:10135000F1CF21E0809709F020E08091E8008E77BE
:101360008093E800CF01C3CF2111C4CFD3CF8091A8
:101370006F03882329F0853069F604C081E0089561
:1013800082E0089583E008956115710529F42091A4
:10139000E8002B772093E8006115710521F1209179
:1013A0006F03222349F1253049F12091E80023FD04
:1013B0001FC02091E80022FFF2CFFC01CF01209155
:1013C000F200222321F38091F1008193CF0161503B
:1013D00071096115710591F7DACF80916F03882348
:1013E00059F0853059F08091E80080FFF6CF02C0B7
:1013F00081E0089580E0089582E0089583E00895F3
:1014000020917603309177032617370748F061154E
:10141000710539F42091E8002E772093E80001C08F
:10142000B90120E061157105D9F130916F033323C3
:1014300009F442C0353009F441C03091E80033FD71
:1014400039C03091E80032FF06C08091E80082FF89
:101450002AC080E008953091E80030FFE3CF20916A
:10146000F20030E0FC01281B390BC9018E0F9F1FD1
:101470006115710551F08032910538F484918093A3
:10148000F100319661507109F0CF21E0809709F0A9
:1014900020E08091E8008E778093E800CF01C2CFF2
:1014A0002111C3CFD2CF80916F03882329F08530DB
:1014B00061F604C081E0089582E0089583E0089514
:1014C000982F953058F59093E900981739F070915E
:1014D000EC002091ED005091F00003C0242F762FF6
:1014E00050E021FF19C03091EB003E7F3093EB00BC
:1014F0003091ED003D7F3093ED003091EB00316095
:101500003093EB007093EC002093ED005093F000CB
:101510002091EE0027FF07C09F5FD3CF8F7080938D
:10152000E90081E0089580E008950F931F93CF9321
:10153000DF93062FEC0110E0101769F198819923D1
:1015400039F12C81E981FA816B81892F8F70853087
:1015500010F080E021C0223010F056E001C052E0CF
:1015600028E030E040E02E173F0720F44F5F220FC5
:10157000331FF9CF4295407F452B991F9927991F1B
:101580006295660F660F607C692B9ADF882309F3EA
:101590001F5F2596D1CF81E0DF91CF911F910F91F1
:1015A00008958091700387FD05C08091E80080FF59
:1015B0000EC012C08091E80082FD05C080916F03CB
:1015C0008111F8CF08958091E8008B7708C0809151
:1015D0006F038111EACF08958091E8008E778093A0
:1015E000E80008958091E4009091E50045E620919F
:1015F000EC0020FF21C02091E80020FD21C02091B7
:101600006F03222389F0253089F02091EB0025FD1E
:101610000FC02091E4003091E5002817390739F315
:10162000415041F0C901E3CF82E0089583E008957D
:1016300081E0089584E008952091E80022FFDFCF43
:1016400080E008953FD041D08091D8008F7780937B
:10165000D8008091D80080688093D8008091D8000D
:101660008F7D8093D80084E089BD86E089BD09B470
:1016700000FEFDCF10926F0310926C0310926D0369
:1016800042E260E080E01CDF8091E1008E7F809389
:10169000E1008091E20081608093E2008091E200AD
:1016A00088608093E2008091E0008E7F8093E0006C
:1016B0000895E3E6F0E080818E7F808381E080936F
:1016C0006E03C0CF1092E20008951092E1000895D9
:1016D0001F920F920FB60F9211242F933F934F93A7
:1016E0005F936F937F938F939F93AF93BF93EF938A
:1016F000FF938091E10082FF0BC08091E20082FFA6
:1017000007C08091E1008B7F8093E1000E947A0105
:101710008091E10080FF17C08091E20080FF13C03C
:101720008091E2008E7F8093E2008091E2008061F0
:101730008093E2008091D80080628093D80019BC29
:1017400010926F03AED18091E10084FF2DC0809193
:10175000E20084FF29C084E089BD86E089BD09B428
:1017600000FEFDCF8091D8008F7D8093D8008091BE
:10177000E1008F7E8093E1008091E2008F7E809374
:10178000E2008091E20081608093E20080916C032E
:10179000811104C08091E30087FF02C084E001C092
:1017A00081E080936F037DD18091E10083FF22C0AF
:1017B0008091E20083FF1EC08091E100877F8093CB
:1017C000E10082E080936F0310926C038091E1004E
:1017D0008E7F8093E1008091E2008E7F8093E20013
:1017E0008091E20080618093E20042E260E080E06C
:1017F00067DE57D1FF91EF91BF91AF919F918F918C
:101800007F916F915F914F913F912F910F900FBEFC
:101810000F901F9018951F93CF93DF93CDB7DEB72E
:10182000AA970FB6F894DEBF0FBECDBFE0E7F3E096
:101830008091F100819323E0E837F207C9F70E9415
:101840006E018091E80083FF14C1209170033091F4
:101850007103832F90E08A30910508F00AC1FC01E2
:10186000E65AFF4F4DC3203881F0223809F001C1FC
:10187000809174038F708093E9008091EB0085FB69
:10188000882780F91092E90004C080916D038111CE
:1018900082E09091E800977F9093E8008093F100B8
:1018A0001092F100C2C0822F8D7F09F0E2C0222386
:1018B00019F0223061F0DDC080917203813009F0AF
:1018C000D8C0333009F080E080936D0328C0809148
:1018D0007203811124C0209174032F7009F4C9C0D0
:1018E0002093E9008091EB0080FF19C08091EB000C
:1018F000333011F4806211C080618093EB0081E08D
:1019000090E0022E01C0880F0A94EAF78093EA0063
:101910001092EA008091EB0088608093EB001092B7
:10192000E9008091E800877F83C02111A2C0109157
:1019300072031F778091E3008078812B8093E3000E
:101940008091E800877F8093E8002BDE8091E8009B
:1019500080FFFCCF8091E30080688093E300112337
:1019600011F083E001C082E080936F0382C02058B1
:10197000223008F07EC080917203909173038C3DF9
:1019800023E0920771F583E08A838AE289834FB767
:10199000F894DE01139620E03EE051E2E32FF0E000
:1019A00050935700E49120FF03C0E295EF703F5F32
:1019B000EF708E2F90E0EA3010F0C79601C0C0960D
:1019C0008D939D932F5F243149F74FBF8091E8009D
:1019D000877F8093E8006AE270E0CE01019675DCB3
:1019E00013C0AE014F5F5F4F609174030E944102CC
:1019F000009709F43EC02091E800277F2093E8007B
:101A0000BC0189819A81FCDC8091E8008B7780930E
:101A1000E8002FC0203869F58091E800877F809327
:101A2000E80080916C038093F1008091E8008E774C
:101A30008093E800B6DD1DC021111BC09091720398
:101A40009230B8F48091E800877F8093E80090930B
:101A50006C03A7DD80916C03811104C08091E300C9
:101A600087FF02C084E001C081E080936F030E9481
:101A70005C018091E80083FF0AC08091E800877FC5
:101A80008093E8008091EB0080628093EB00AA963F
:101A90000FB6F894DEBF0FBECDBFDF91CF911F917F
:101AA00008950895CF9380916F038823A9F08091C2
:101AB000E9008F709091EC0090FF02C090E801C0A7
:101AC00090E0C92FC82B1092E9008091E80083FDB7
:101AD000A2DECF70C093E900CF9108956F927F92FC
:101AE0008F929F92AF92BF92CF92DF92EF92FF922E
:101AF0000F931F93CF93DF9300D01F92CDB7DEB724
:101B00007C01ADB6BEB68091E80083FF00C1F7014D
:101B1000808190E020917403309175032817390774
:101B200009F0F5C080917103833009F497C030F457
:101B3000813071F0823009F4CEC0E9C08A3009F4F6
:101B4000B2C08B3009F49BC0893009F0E0C048C0B6
:101B500080917003813A09F0DAC08DB69EB61A8280
:101B6000198280917203109173038B83F701408572
:101B700050E08DB79EB7841B950B0FB6F8949EBFAF
:101B80000FBE8DBFEDB7FEB731966F0160E070E01C
:101B9000CF01D2D14FEF410F8E010F5F1F4F960142
:101BA000BE016D5F7F4FC7010E949C01F7018681D6
:101BB0009781009721F0408550E0B601B4D1109292
:101BC000E9008091E800877F8093E80069817A814D
:101BD000C6017BDB8091E8008B778093E80038C0FA
:101BE00080917003813209F092C08DB69EB600914B
:101BF00076031091770370907203609073038DB732
:101C00009EB7801B910B0FB6F8949EBF0FBE8DBF81
:101C1000EDB7FEB731966F018091E800877F809322
:101C2000E800B801CF01B0DB8091E8008E778093A7
:101C3000E80021E0711001C020E030E0021B130B2E
:101C40002C0D3D1D4FEF460D672DC7010E94BE01B3
:101C50000FB6F8949EBE0FBE8DBE59C08091700322
:101C6000813A09F054C08091E800877F8093E800B2
:101C70008091E80080FFFCCFF701818540C0809112
:101C80007003813209F043C08091E800877F809320
:101C9000E80087DC9091720381E0911101C080E03F
:101CA000F701818734C080917003813281F5809182
:101CB000E800877F8093E80074DC80917203909144
:101CC0007303882736E0969587953A95E1F7F701F3
:101CD000958784871CC080917003813AC1F48091FC
:101CE000E800877F8093E8008091E80080FFFCCFC8
:101CF000F701848595859695879596958795809328
:101D0000F1008091E8008E778093E8004ADC0FB6FE
:101D1000F894BEBE0FBEADBE0F900F900F90DF9136
:101D2000CF911F910F91FF90EF90DF90CF90BF90D8
:101D3000AF909F908F907F906F900895FC0139969F
:101D400027E0DF011D922A95E9F721E0FC012187B8
:101D500024EF31E03587248723E0248361E0019676
:101D6000E4CB5F926F927F928F929F92AF92BF92DD
:101D7000CF92DF92EF92FF920F931F93CF93DF9357
:101D800000D01F92CDB7DEB77C01ADB6BEB6809154
:101D90006F03843009F08BC08091E4009091E500DE
:101DA000F701228533852817390709F480C081811E
:101DB0008F708093E9008091E80085FF78C08DB630
:101DC0009EB6408550E08DB79EB7841B950B0FB62D
:101DD000F8949EBF0FBE8DBFEDB7FEB731966F0171
:101DE0001B821A82198260E070E0CF01A5D08E01BB
:101DF0000F5F1F4F960140E0BE016D5F7F4FC7012F
:101E00000E949C01682EF70184859585892B41F0FD
:101E100021E086859785892B09F020E0722E01C08C
:101E2000712CF701068117810115110589F049818F
:101E30005A81B801C6016AD055245394892B09F4FC
:101E4000512CF701408550E0B601C8016CD001C0AB
:101E5000512C29813A81232BF1F0611004C05110DB
:101E600002C070FE18C0F701848595859787868724
:101E700081818F708093E9008B8181118093F100C3
:101E800069817A8140E050E0C601D7D98091E800AD
:101E90008E778093E8008091E4009091E500F7014F
:101EA000938782870FB6F8949EBE0FBE8DBE0FB685
:101EB000F894BEBE0FBEADBE0F900F900F90DF9195
:101EC000CF911F910F91FF90EF90DF90CF90BF9037
:101ED000AF909F908F907F906F905F9008950024B7
:101EE000552704C0080E591F880F991F009729F025
:101EF00076956795B8F37105B9F7802D952F0895FC
:101F0000EE0FFF1F0590F491E02D0994FB01DC0119
:101F100004C08D910190801921F441505040C8F7C0
:101F2000881B990B0895FB01DC0102C001900D9202
:101F300041505040D8F70895DC0101C06D934150E5
:101F40005040E0F70895DC01CB01FC01F999FECF88
:101F500006C0F2BDE1BDF89A319600B40D92415031
:101F60005040B8F70895F999FECF92BD81BDF89A17
:101F7000992780B50895DC01A40FB51F415050404A
:101F800040F0CB01840F951F2E9105D04150504059
:101F9000D8F70895262FF999FECF92BD81BDF89A02
:101FA000019700B4021639F01FBA20BD0FB6F8949D
:0C1FB000FA9AF99A0FBE0895F894FFCF3A
:101FBC000282190000015601190000000000000007
:101FCC000183080000016F01080000000000000000
:101FDC0000810800000177010800000000000000EB
:101FEC0050020200182520BE58027A019A012601DF
:101FFC003F0158011003F401AC021003F401AC02D0
:06200C00302E362E3100DB
:00000001FF
